:020000040800F2
:100000004807002089260008690F00086B0F0008C8
:100010006F0F0008730F0008770F00080000000042
:100020000000000000000000000000007B0F00083E
:100030007D0F0008000000007F0F0008810F0008FE
:10004000A3260008A3260008A3260008A32600086C
:10005000A3260008A3260008A3260008A32600085C
:10006000A3260008A3260008A3260008A32600084C
:10007000A3260008A3260008A3260008A32600083C
:10008000A3260008A3260008A3260008A32600082C
:10009000A3260008A3260008A3260008A32600081C
:1000A000A3260008A3260008A3260008A32600080C
:1000B000A326000809160008A3260008A3260008A6
:1000C000A3260008A3260008A3260008A3260008EC
:1000D000A3260008FD250008A32600087D120008BD
:1000E000A3260008A3260008A3260008DFF80CD0EA
:1000F00004F0BEFD00480047210F0008480700201B
:10010000F0B58FB0FA480068002836D1F948406948
:10011000F8490969F74AD268CDE900210290F5480B
:100120008368F5A1426807A804F002FE102307AA1D
:100130000021084601F03BFFF549486C04F00AFB3A
:1001400004460D46F249086804F004FB0646F048F0
:10015000B0F84800CDE902450490ED4840683246C9
:100160000B46ECA1009007A804F0E2FD102307AABB
:100170000221002001F01BFF31E0EC4800680090F4
:10018000E348B0F84830EAA1826807A804F0D0FD3F
:10019000102307AA0021084601F009FFDC4890F867
:1001A0004100DB4991F84010D94A526AD84B1B6A8A
:1001B000CDE90232CDE90410D548C069D449896936
:1001C000CDE90010D2484369DEA1026907A804F016
:1001D000AFFD102307AA0221002001F0E8FE0FB0B6
:1001E000F0BD2DE9F0410027002600240025DEA106
:1001F000DE4804F0A6F9DD49471ADDA1DB4804F02A
:10020000A0F9DA49461A00BF7C1C07E0D748005D18
:10021000303805EB850100EB4105641CB442F5DB89
:100220002846BDE8F08110B5024600200021D14CDF
:100230002488C4F30D0300BF05E0CC4C645C9442F9
:1002400000D10846491C9942F7DB10BD0246002147
:10025000C8480088C0F30D0300BF06E0C348405CF7
:10026000904201D108467047491C9942F6DB0020B4
:10027000F9E72DE9F0418CB08046002600270024E4
:100280000025B9A1B94804F05CF9B849461A2D20F7
:10029000FFF7DCFF0746741C07E0B448005D303808
:1002A00005EB850100EB4105641CBC42F5DB0095C4
:1002B00000252D20FFF7CAFF06462D20FFF7B3FFCC
:1002C0000746741C07E0A948005D303805EB85013E
:1002D00000EB4105641CBC42F5DB019500252D2097
:1002E000FFF7A1FF06462020FFF7B0FF0746741C6A
:1002F00007E09E48005D303805EB850100EB4105C5
:10030000641CBC42F5DB029500252020FFF79EFF10
:1003100006463A20FFF79AFF0746741C07E0934809
:10032000005D303805EB850100EB4105641CBC42E3
:10033000F5DB039500253A20FFF788FF06463A20B3
:10034000FFF771FF0746741C07E08848005D3038EE
:1003500005EB850100EB4105641CBC42F5DB04950F
:1003600000253A20FFF75FFF06462920FFF75BFFD5
:100370000746741C07E07D48005D303805EB8501B9
:1003800000EB4105641CBC42F5DB05953022694653
:10039000404604F0B2F80CB0BDE8F081F0B58DB085
:1003A0007448008800F40040002874D072A16F489F
:1003B00004F0C7F8C0B15648C068401C5449C86032
:1003C0000846C068022801DB0020C8605048C068A9
:1003D00018B96BA004F09CFC06E04D48C0680128E9
:1003E00002D16CA004F094FC70A1604804F0A9F85C
:1003F00088B14748C06818B961A004F089FC0AE0D8
:100400004348C068012803D162A004F081FC02E0E7
:1004100069A004F07DFC6FA1544804F092F830B15B
:10042000FFF7DFFE3A4988606EA004F071FC72A10C
:100430004E4804F086F858B101A8FFF71AFF3022A1
:1004400001A93348103004F058F86EA004F060FCA5
:1004500070A1464804F075F878B1FFF7C2FE2C4948
:10046000A1F848000846B0F84800032802DB022043
:10047000A1F848006AA004F04BFC6DA13B4804F0D1
:1004800060F8C0B1224890F8400028B90120204906
:1004900081F8400004E047E100201D4981F8400058
:1004A0001B4890F8400018B964A004F031FC02E049
:1004B00066A004F02DFC69A12C4804F042F8A0B11C
:1004C000134890F8410020B90120114981F84100FA
:1004D00003E000200E4981F841000D4890F84100EA
:1004E00020B960A004F014FCC7E0C6E0C2E0000040
:1004F00008000020D80100202532642D2532642018
:100500002532643A2532643A253264202000000006
:100510008C01002025302E3266432025644320259F
:10052000302E3266636D2025640000000C00002030
:100530002532644320204C6576656C3A2564202082
:10054000256400002532642D2532642D2532642077
:100550002532643A2532643A25326420543A2564BF
:100560002C483A256400000028000000800200208A
:1005700029000000740100206D6F64656C000000AC
:100580005468652068656174696E67206D6F646585
:100590000D0A000053746572696C697A6174696F41
:1005A0006E206D6F64650D0A000000006765744D74
:1005B0006F64656C000000004865617420707265AE
:1005C000736572766174696F6E206D6F64650D0A74
:1005D0000000000073657454617267657454656D42
:1005E0007000000073657454617267657454656DC2
:1005F00070204F4B210D0A0073657454696D65724C
:100600000000000073657454696D6572204F4B21C2
:100610000D0A00007365744C6576656C000000007F
:100620007365744C6576656C204F4B210D0A000094
:1006300054696D6572466C6167000000436C6F73AE
:10064000652054696D6572210D0A00004F70656E5A
:100650002054696D6572210D0A000000486F7446D0
:100660006C616700436C6F736520486F74210D0ADD
:1006700000000000FBA004F04BFBFDA1FE4803F0CE
:1006800060FF00B3FD49486C04F064F804460D4671
:10069000FA49086804F05EF806460F46F74890F8F5
:1006A0004100F64991F84010CDE90245CDE904102A
:1006B000F2488068F149496832463B46CDE900106E
:1006C000EF4804F025FBEFA1EB4803F03AFF78B1C7
:1006D000EE484069ED490969EC4AD268CDE900214C
:1006E0000290EA48836842680168E9A004F010FBC0
:1006F000EEA1E14803F025FF78B1E048406ADF4908
:10070000096ADE4AD269CDE900210290DB4883699B
:1007100042690169E8A004F0FBFAC821D64803F059
:1007200005FF0020EB4908800DB0F0BD2DE9F04732
:1007300000244FF080450026E74FD048B0F848002D
:10074000012802D1E54D870708E0CC48B0F8480001
:10075000022803D10024E24D0026E04FC749486C2F
:1007600003F0F8FF804632463B4604F007F803D218
:100770000120DC4908602EE0C049486C03F0EAFF24
:10078000804632463B4604F011F80DD8BB49486C10
:1007900003F0E0FF804622462B4603F0EFFF03D232
:1007A0000020D049086016E0B449486C03F0D2FF3D
:1007B000804622462B4603F0F9FF0CD20120C9499E
:1007C0000C390860642001F07CFE0020C649C1F8A5
:1007D000A001C4490860A949486C4FF07E5104F05B
:1007E00019F814D2A54890F8420080B10120BF4901
:1007F00008600020BE49C1F8BC01642001F061FE20
:100800000020BA4908600120B949C1F8BC01BDE81F
:10081000F08710B599498968481E03F06EFF0446B9
:1008200096480168204603F0FFFF08D8002093494E
:1008300081F84000012081F841000020C86010BD0F
:1008400010B50020A94908310860642001F039FE84
:100850000120A749C1F8BC0110BD012087494969A1
:100860008A4A5268914201D000201EE0834989697A
:10087000864A9268914201D0002016E07F49C969FA
:10088000824AD268914201D000200EE07B49096A79
:100890007E4A1269914201D0002006E07749496AF8
:1008A0007A4A5269914200D0002070472DE9F04108
:1008B0000546724845608F48007B00282DD06F4860
:1008C00090F84200002828D08A4800686F49C9681B
:1008D000884222D1874840686C49096988421CD106
:1008E0008448806869494969884216D1634A116819
:1008F000804A106903F089FE804603F02BFF06460C
:1009000021F00041022808DC00207849091D086018
:100910007849087378A004F0FBF9584890F8400033
:10092000002849D0FFF799FF0446002C33D07148C6
:10093000007B00282FD17CA004F0EAF9FFF780FFAC
:1009400001206A49091D08606A4908734F48C06858
:1009500008604E48006948604C48406988604748D4
:100960000068086108464068401C486008464068C6
:100970003B282ADD084640683C3848600846006845
:10098000401C08600846006817281EDD08460068FD
:100990001838086019E03CB95648007B20B900209F
:1009A0005249091D086010E0344890F8420060B9CF
:1009B00000205049087308E000204E4908732F4872
:1009C00090F841004949091D08602C49486C4FF0D6
:1009D0007E5103F01FFF09D3284603F08EFE064622
:1009E00026480168304603F015FF1BD100203F491F
:1009F000091D08603F4908732049486C4FF07E513B
:100A000003F008FF02D20120BDE8F081284603F080
:100A100074FE064619480168304603F0FBFE01D813
:100A20000220F1E70020EFE710B544480078B8B99C
:100A30001E20FFF73BFF022813D1502140A004F0F5
:100A400067F90020294908310860642001F039FD68
:100A500001202749C1F8BC010848806807497DE0AA
:100A600083E0A0E04F70656E20486F74210D0A008E
:100A7000676574496E666F00800200208C0100205B
:100A80004C5E000867657454696D6500D8010020EC
:100A900054696D653A20323025642D25642D256416
:100AA0002025643A25643A25640D0A00676574546C
:100AB000696D65720000000054696D65723A202509
:100AC000642D25642D25642025643A25643A256427
:100AD0000D0A0000740100200000F03F00000840F3
:100AE00000001040AC01214200002142B40122422A
:100AF00000002242080200204E6F206368616E678A
:100B00006520696E2074656D7065726174757265BB
:100B10002C205475726E206F66662068656174695A
:100B20006E670D0A0000000054696D6520746F2027
:100B300068656174207570210D0A000010000020A6
:100B40005468652074656D70657261747572652096
:100B5000726561636865643A25640000486002203C
:100B6000C8600120F94908701DE00020F84981F8AB
:100B7000400081F841008868FFF798FE022812D1F2
:100B8000F3488168AFF2480004F0C2F80020F14950
:100B90000860642001F095FC0120EF49C1F8BC0118
:100BA0000220EB49C86010BD10B5E9498868FFF71D
:100BB0007DFE022812D1E6488168AFF27C0004F085
:100BC000A7F80020E3490860642001F07AFC0120C6
:100BD000E149C1F8BC010220DD49C86010BDDF4910
:100BE0000968012900D07047DD490968082911D238
:100BF000DFE801F004111D2A3D506376D44989686D
:100C00000A2907DAD249896801EB810100EB410129
:100C1000CF4A916077E0CE4AA2F848001146B1F879
:100C20004810032902DB0221A2F848106BE0C849F2
:100C300009690A2907DAC649096901EB810100EB54
:100C40004101C34A11615EE0C14949690A290DDACF
:100C5000BF49496901EB810100EB4102BC494A618E
:100C600049690C2902DD0C22B9494A614BE0B849B7
:100C700089690A290DDAB649896901EB810100EB1E
:100C80004102B3498A6189691F2902DD1F22B049E7
:100C90008A6138E0AE49C9690A290DDAAC49C969E7
:100CA00001EB810100EB4102A949CA61C969172919
:100CB00002DD1722A649CA6125E0A549096A0A2969
:100CC0000DDAA349096A01EB810100EB4102A04959
:100CD0000A62096A3B2902DD3B229D490A6212E051
:100CE0009B49496A0A290DDA9949496A01EB810150
:100CF00000EB410296494A62496A3B2902DD3B22E8
:100D000093494A6200BF00BF00BF6CE79348006888
:100D1000012800D0704792480068082847D2DFE8D1
:100D200000F0040C161E262E363E894880680A21E3
:100D300090FBF1F08649886039E08548B0F84800BA
:100D40000A2190FBF1F08249A1F848002FE0804889
:100D500000690A2190FBF1F07D49086127E07C4899
:100D600040690A2190FBF1F1794841611FE0784820
:100D700080690A2190FBF1F17548816117E07448A0
:100D8000C0690A2190FBF1F17148C1610FE0704820
:100D9000006A0A2190FBF1F16D48016207E06C489E
:100DA000406A0A2190FBF1F16948416200BF00BF2F
:100DB00000BFAFE710B5102401F037FA0446A4F1E4
:100DC0000B0005283CD2DFE800F03803101C2A0095
:100DD0006248006818B901206049086002E00020FC
:100DE0005E49086001F009F836E05D480068401C83
:100DF0005B49086008460068082801DB002008609D
:100E00002AE0534890F8410020B90120504981F868
:100E1000410003E000204E4981F841001CE04C48AD
:100E200090F8400020B90120494981F8400003E0D2
:100E30000020474981F840000EE0FFF767FF0BE014
:100E40004648006808B1102C00D105E00A2C02DAEF
:100E50002046FFF7C4FE00BF00BF10BD2DE9F047DC
:100E6000FFF7A8FF3D48006800283AD100F004FDD4
:100E70000A2190FBF1F5284603F03FFC3449086055
:100E80000A21012000F079FB8146484603F03EFC30
:100E9000824603F05FFC07460022134603F0BBFBCB
:100EA000054603F09BFC0446294844642948001F7A
:100EB0000068274981F842000846C06810B9FFF76A
:100EC00073FE0CE02248C068012802D1FFF7ACFD98
:100ED00005E01F48C068022801D1FFF79AFCFFF720
:100EE00025FCBDE8F08710B501F0AEFA4FF4A06024
:100EF00002F060F94FF4E13001F034FB00F056F9F4
:100F000000F030F900F09DFC00F0DEFA01F0DEF8B0
:100F100001F06AF9134800F02AFE00F06EFF10BDE0
:100F2000FFF7E1FF4FF47A7001F0CBFA0120094995
:100F300008600AE0FFF792FFFFF730FA00F03AFE90
:100F4000FFF7DEF8C82001F0BCFAF3E7100000203C
:100F50008C010020BC012242000022420800002037
:100F60000C00002000000020704700BFFEE700BF1B
:100F7000FEE700BFFEE700BFFEE77047704770471F
:100F8000704700000CB50020019000906C4800688C
:100F900040F480306A49086000BF6948006800F486
:100FA000003000900198401C0190009818B90198F9
:100FB000B0F5A06FF1D16248006800F4003010B1C4
:100FC0000120009001E0002000900098012843D10A
:100FD0005C48006840F010005A4908600846006804
:100FE00020F0030008600846006840F00200086036
:100FF000534840685249486008464068486008467F
:10100000406840F4806048600846406820F47C10E6
:1010100048600846406840F4E810486008460068A8
:1010200040F08070086000BF4548006800F0007024
:101030000028F9D04248406820F003004049486049
:101040000846406840F00200486000BF3C484068E5
:1010500000F00C000828F9D10CBD10B5FFF792FF85
:1010600010BD10B53648006840F0010034490860F2
:1010700008464068344908403149486008460068DD
:10108000324908402E4908600846006820F4802054
:1010900008600846406820F4FE0048604FF41F00D6
:1010A0008860FFF7DAFF4FF000602949086010BD43
:1010B00010B5002100200022214B5B6803F00C01D9
:1010C00021B1042906D0082928D107E0214B224C60
:1010D000236027E01F4B204C236023E0184B5B6804
:1010E00003F47010164B5B6803F48032022303EBA9
:1010F000904022B9194B4343174C23600DE0104B2D
:101100005B6803F4003323B1144B4343124C236058
:1011100003E0104B4343104C236003E00D4B0E4C97
:10112000236000BF00BF064B5B68C3F303130C4C86
:10113000E15C094B1B68CB40074C236010BD0000ED
:1011400000100240002002400000FFF8FFFFF6FE02
:1011500008ED00E000127A001400002000093D00B4
:101160001800002008B50121142001F0BBFD4FF448
:101170000040ADF8000010208DF8030003208DF82A
:1011800002006946134801F0F1FA4FF40050ADF83F
:10119000000069460F4801F0E9FA4FF41060ADF81D
:1011A000000069460C4801F0E1FA08BD08B50121CC
:1011B000102001F097FD4FF4C040ADF80000102062
:1011C0008DF8030003208DF802006946014801F004
:1011D000CDFA08BD001001400008014010B586B0EE
:1011E00004460121082001F07DFD0121880401F061
:1011F00086FD4FF48060ADF8140003208DF81600D2
:1012000018208DF8170005A9874801F0AFFA4FF4B0
:101210000060ADF8140004208DF8170005A982487D
:1012200001F0A4FA27208DF8000000208DF80100BD
:1012300003208DF8020001208DF80300684601F0BC
:10124000BEFF01940020ADF80800ADF80A00ADF82B
:101250000C00ADF810000C20ADF80E0001A9734889
:1012600001F0E7FD012240F22551704801F079FEBE
:1012700001216E4801F069FE06B010BD10B50024D2
:101280006A4801F0D3FEC4B269486A4909784454F7
:1012900068480078401C6749087008460078642850
:1012A00001DB0020087010BD002004E00021604A2E
:1012B0001154411C88B26428F8DB00215D4A11708A
:1012C000704710B504460BE000BF4021574801F0BD
:1012D00017FF0028F9D014F8011B544801F0A2FEB2
:1012E00020780028F0D110BD10B50446FFF7DCFFD0
:1012F0002046FFF7E6FF50A0FFF7E3FF10BD10B553
:10130000044621464A4803F01CF908B1012010BDEB
:101310000020FCE72DE9F04180460C4615461E46AC
:1013200000270EE04046FFF7DFFFB0B201F0C9F83A
:101330002046FFF7E4FF10B10120BDE8F081781CE2
:10134000C7B2AF42EEDB0020F7E710B564230322FB
:101350003AA13BA0FFF7DEFF04464FF4167001F000
:10136000B0F814B94FF0FF3010BD6423032233A14D
:1013700035A0FFF7CFFF04464FF4167001F0A1F837
:1013800014B96FF00100EFE7642303222BA132A010
:10139000FFF7C0FF04464FF4167001F092F814B93D
:1013A0006FF00200E0E76423032224A132A0FFF7DC
:1013B000B1FF04464FF4167001F083F814B96FF0D2
:1013C0000300D1E7642303221CA12FA0FFF7A2FF93
:1013D00004464FF4167001F074F814B96FF004006D
:1013E000C2E76423032215A12DA0FFF793FF044653
:1013F0004FF4167001F065F814B96FF00500B3E70B
:101400000020B1E710B504463223032228A129A009
:10141000FFF780FFC82001F054F82046FFF751FF86
:10142000642001F04EF810BD000C0140004800405F
:101430001C020020280000200D0000004F4B00007F
:1014400041540D0A0000000041542B43574D4F44B6
:10145000453D320D0A00000041542B435753415083
:101460003D225A48222C223132333435363738392E
:10147000222C352C330D0A0041542B4349504D5535
:10148000583D310D0A00000041542B43495053454B
:10149000525645523D312C353030300D0A00000097
:1014A00041542B43495053544F3D300D0A00000026
:1014B0003E00000041542B43495053454E443D30BB
:1014C0002C31340D0A00000000B587B001214FF423
:1014D000017001F007FC4FF4004001F067FB0220AF
:1014E000ADF8040000208DF8070001A92E4801F096
:1014F0003DF92E4801F0CCFE002002908DF80C0042
:101500008DF80D004FF4602004900020059001201C
:101510008DF8180002A9254801F0E1FE01212348B9
:1015200001F009FF214801F028FF00BF1F4801F02A
:1015300029FF0028FAD11D4801F02EFF00BF1B48EB
:1015400001F02FFF0028FAD107B000BD10B5044606
:10155000072301222146154801F059FF01211348B4
:1015600001F029FF00BF0221104802F095F8002881
:10157000F9D00E4801F0B2FF10BD2DE9F041074649
:101580000C460025002608E03846FFF7DFFF05443B
:10159000052000F096FF701CC6B2A642F4DBB5FB36
:1015A000F4F080B2BDE8F081000801400024014061
:1015B0007FB505460C460121022001F0A0FBADF8E5
:1015C0000850ADF804400020ADF80A00ADF8060060
:1015D00001A9334802F058F901221146304802F0BF
:1015E000CAFC1D208DF8000003208DF801008DF845
:1015F000020001208DF80300684601F0E0FD0121A2
:10160000274802F09DFC7FBD10B50121244802F05F
:1016100060FF18B10121224802F06CFF10BD30B507
:1016200089B005460C460121022001F068FB01212A
:10163000092001F057FB01211A4801F068F9022046
:10164000ADF8200018208DF8230003208DF822002B
:1016500008A9154801F08AF8ADF81850ADF8144003
:101660000020ADF81A00ADF8160005A90C4802F0EC
:101670000BF97020ADF804000120ADF80600002041
:10168000ADF80C0001A9064802F07DF908210448D4
:1016900002F08FFD0121024802F052FC09B030BD7A
:1016A0000004004000081A00000C014010B59448E6
:1016B000006820F00F00924908600846006840F07A
:1016C0000300086000208F49086040F2EE2000F01F
:1016D000D4FE01208C49C1F880010F2000F0CDFE1E
:1016E00010BD10B500248648006820F00F00844922
:1016F00008600846006840F00800086004E0601CCC
:10170000C4B2012000F0B9FE7E488038006808B1FC
:10171000C82CF4DBC82C01DB012010BD002404E040
:10172000601CC4B2012000F0A8FE76488038006832
:1017300008B9F02CF4DBF02C01DB0120EDE70020F0
:10174000EBE710B56E48006820F00F006C490860A8
:101750000846006840F003000860002069490860FE
:10176000022000F08AFE01206749C1F88001644828
:10177000006820F00F00624908600846006840F0E9
:10178000080008600C2000F078FE5E488038006891
:1017900008B1012400E00024322000F06EFE204653
:1017A00010BD70B50026012508E0FFF7CAFF04460A
:1017B000E00140EA6600C6B2681CC5B2082DF4DD3F
:1017C000304670BD70B504464D48006820F00F00EB
:1017D0004B4908600846006840F003000860012596
:1017E00020E004F0010664106EB100204549086055
:1017F000022000F042FE01204349C1F880013C2054
:1018000000F03BFE0CE000203E4908603C2000F068
:1018100034FE01203C49C1F88001022000F02DFE79
:10182000681CC5B2082DDCDD70BD10B5FFF73EFFAA
:10183000FFF757FFCC20FFF7C5FF4420FFF7C2FF9B
:1018400010BD08B50121042001F04CFA0120ADF8CB
:10185000000010208DF8030003208DF80200694677
:10186000274800F083FF0121254801F02CF8FFF7FD
:101870001DFFFFF736FF08BD2DE9F84FFFF7D5FF35
:10188000FFF714FFFFF72DFFCC20FFF79BFFBE20D3
:10189000FFF798FFFFF785FF8346FFF782FF0446B7
:1018A000072C08DDE043C4B26FEA0B0000F0FF0B29
:1018B0004FF0000A01E04FF0010AA1464FEA09206B
:1018C0000FFA80F909EB0B000FFA80F9484602F095
:1018D00014FF009002F03EFF074600220B4B02F07F
:1018E0009AFE054602F017FF0FFA80F9BAF1000FD1
:1018F00002D04846BDE8F88FC9F1000000B2F9E710
:101900000008014080012142000021420000E43F24
:1019100008B50121082001F0E5F9E020ADF800004C
:1019200003208DF8020010208DF803006946B148AD
:1019300000F01CFF08BD38B50446012C0DD1402035
:10194000ADF8000003208DF8020010208DF8030090
:101950006946A84800F00AFF0DE064B94020ADF8E0
:10196000000003208DF8020048208DF8030069462E
:10197000A04800F0FBFE38BD07E06E2101E04A1EE2
:10198000D1B20029FBDC421ED0B20028F5DC704742
:10199000F0B504460D4626462F4680209549103165
:1019A0000860002319E006F0010020B140209149B1
:1019B0001031086003E040208E4914310860761031
:1019C00020208C49103108600220FFF7D5FF20202D
:1019D000884914310860581CC3B2082BE3DB00238C
:1019E00019E007F0010020B1402082491031086061
:1019F00003E040207F49143108607F1020207D499A
:101A0000103108600220FFF7B7FF20207949143118
:101A10000860581CC3B2082BE3DB802075491431E1
:101A20000860F0BD2DE9F047064637468020714931
:101A300010310860002519E007F0010020B14020B6
:101A40006C491031086003E040206A491431086095
:101A50007F1020206749103108600220FFF78CFFBB
:101A60002020644914310860681CC5B2082DE3DBEE
:101A70000020FFF760FF002517E0641040215D485B
:101A800000F007FF10B144F0800401E004F07F048F
:101A900020205849103108600220FFF76DFF2020F8
:101AA000544914310860681CC5B2082DE5DB80205C
:101AB0005049143108600120FFF73DFF2046E1172F
:101AC00004EB1171C1F30718E11704EB117109114F
:101AD000A4EB011101F0FF0908EB880009EB4000BD
:101AE00000F0FF0A5046BDE8F08710B5044600211B
:101AF0008E20FFF74DFF61798020FFF749FF2179A4
:101B00008220FFF745FFE1788420FFF741FFA178AD
:101B10008620FFF73DFF61788820FFF739FF2178A5
:101B20008C20FFF735FF80218E20FFF731FF10BD9D
:101B300010B58120FFF776FF044600218E20FFF7C5
:101B400027FF44F0800421468020FFF721FF10BDCD
:101B500010B58120FFF766FF044600218E20FFF7B5
:101B600017FF00BF21468020FFF712FF10BD10B500
:101B70000446FFF7CDFE0220FFF7FEFE80201D4940
:101B8000143108602020086000218E20FFF700FF3C
:101B9000A7219020FFF7FCFE80218E20FFF7F8FEA2
:101BA0008120FFF73FFF00F0800010B12046FFF7D3
:101BB0009CFF10BD10B58D20FFF734FF0E49086063
:101BC0008920FFF72FFF0C4948608720FFF72AFF85
:101BD000094988608520FFF725FF0749C8608320F1
:101BE000FFF720FF044908618120FFF71BFF02492E
:101BF000486110BD000C0140D801002010B54FF421
:101C00000051F94800F05FFE4FF40041F64800F043
:101C10005AFE4FF40041F44800F057FE4FF40051D3
:101C2000F14800F052FE10BD10B54FF40051EE48DF
:101C300000F049FE4FF40041EB4800F046FE4FF43F
:101C40000041E94800F03FFE10BD10B54FF40051CF
:101C5000E54800F038FE4FF40051E34800F035FE4F
:101C600010BD2DE9F04105462C464FF40051DE48E9
:101C700000F02BFE00261CE0274607F08007802F8F
:101C800004D13902D84800F01EFE04E04FF40041B0
:101C9000D54800F01AFE6006040E4FF40051D248F9
:101CA00000F011FE4FF40051CF4800F00EFE701C02
:101CB000C6B2082EE0DBBDE8F08110B50446FFF7A0
:101CC0009DFF7820FFF7CDFFFFF7BFFF0020FFF754
:101CD000C8FFFFF7BAFF2046FFF7C3FFFFF7B5FFC6
:101CE000FFF7A2FF10BD10B50446FFF787FF78206D
:101CF000FFF7B7FFFFF7A9FF4020FFF7B2FFFFF79D
:101D0000A4FF2046FFF7ADFFFFF79FFFFFF78CFF13
:101D100010BD70B504460D461DB1E0B2FFF7E3FFFC
:101D200002E0E0B2FFF7C9FF70BD70B506460024BF
:101D300018E004F1B0000021FFF7EBFF0021084696
:101D4000FFF7E7FF00211020FFF7E3FF002505E084
:101D500001213046FFF7DDFF681CC5B2802DF7DB9F
:101D6000601CC4B2082CE4DB70BD06E041F66501DE
:101D700000E0491E0029FCD1401E0028F6D1704722
:101D8000014605E0002001E0421CD0B27B28FBDBCD
:101D90000A1EA1F10101F5D1704770B504460D4648
:101DA00005F1B0000021FFF7B4FF102141EA141043
:101DB0000021FFF7AEFF04F00F000021FFF7A9FF9D
:101DC00070BD10B500218D20FFF7A3FF0021142066
:101DD000FFF79FFF0021AF20FFF79BFF10BD10B55D
:101DE00000218D20FFF795FF00211020FFF791FFC4
:101DF0000021AE20FFF78DFF10BD70B5002418E064
:101E000004F1B0000021FFF784FF00210846FFF72E
:101E100080FF00211020FFF77CFF002505E0012155
:101E20000020FFF776FF681CC5B2802DF7DB601C31
:101E3000C4B2082CE4DB70BD70B5002418E004F1D6
:101E4000B0000021FFF765FF00210846FFF761FFA2
:101E500000211020FFF75DFF002505E00121084665
:101E6000FFF757FF681CC5B2802DF7DB601CC4B2BA
:101E7000082CE4DB70BD2DE9F04707460E4690467E
:101E8000994600250024A8F12000C5B27F2F02DD6D
:101E90000027B01CC6B2B9F1100F24D13146384624
:101EA000FFF77BFF002408E004EB05114F4A505C6C
:101EB0000121FFF72EFF601CC4B2082CF4DB701C5C
:101EC000C1B23846FFF769FF002409E004EB0511B1
:101ED0000831464A505C0121FFF71BFF601CC4B269
:101EE000082CF3DB12E031463846FFF756FF00249A
:101EF0000AE005EB45013E4A02EB4101085D012184
:101F0000FFF707FF601CC4B2062CF2DBBDE8F087C8
:101F100010B50246012000E050430B1EA1F1010460
:101F2000E1B2F9D110BD2DE9FF5F074691461E468B
:101F30000E9D4FF0000A002435E0301B401EC1B258
:101F40000A20FFF7E5FFB9FBF0F00A21B0FBF1F240
:101F500001FB1208BAF1000F14D1701EA04211DD6E
:101F6000B8F1000F0CD1AB4605EBDB71491001FB5A
:101F70000471C8B22B4620220199FFF77CFF10E0C4
:101F80004FF0010AAB4605EBDB71491001FB047110
:101F9000C8B208F13001CAB22B460199FFF76BFFB6
:101FA00000BF601CC4B2B442C7DBBDE8FF9F2DE98F
:101FB000F04104460F461546984600260FE0AA5DFC
:101FC000434639462046FFF756FF04F10800C4B2E5
:101FD000782C02DD0024B81CC7B2701CC6B2A85D04
:101FE0000028ECD1BDE8F081000C01405C580008ED
:101FF000345600082DE9F04180460E46154600276C
:1020000031464046FFF7C9FE00240AE0744A02EB5D
:102010008511085D0121FFF77CFE781CC7B2601CAA
:10202000C4B2102CF2DB701CC1B24046FFF7B5FE03
:1020300000240CE06900491C694A02EB4111085D6B
:102040000121FFF766FE781CC7B2601CC4B2102CD9
:10205000F0DBBDE8F0812DE9F05F06460F469046C3
:102060001C46DDF828A04FF0000BE11704EB51717E
:10207000C910A4EBC10131B92046E11704EB51713D
:10208000C1F3C70506E02046E11704EB5171C91002
:10209000491CCDB23D4615E029463046FFF77DFE8E
:1020A000B1460BE059460BF1010B1AF80100012172
:1020B000FFF72FFE09F1010000F0FF09C145F1DB38
:1020C000681CC5B2A542E7DBBDE8F09F08B5012159
:1020D000082000F007FE4FF42040ADF8000010206B
:1020E0008DF8030003208DF8020069463D4800F09A
:1020F0003DFB4FF420413B4800F0E5FB4FF44870B6
:1021000000F0DFF90021AE20FFF703FE00210846B2
:10211000FFF7FFFD00211020FFF7FBFD002140200D
:10212000FFF7F7FD0021B020FFF7F3FD002181202C
:10213000FFF7EFFD0021FF20FFF7EBFD0021A120BD
:10214000FFF7E7FD0021A620FFF7E3FD0021A8200F
:10215000FFF7DFFD00213F20FFF7DBFD0021C82056
:10216000FFF7D7FD0021D320FFF7D3FD002108465C
:10217000FFF7CFFD0021D520FFF7CBFD0021802008
:10218000FFF7C7FD0021D820FFF7C3FD0021052080
:10219000FFF7BFFD0021D920FFF7BBFD0021F12093
:1021A000FFF7B7FD0021DA20FFF7B3FD0021122071
:1021B000FFF7AFFD0021DB20FFF7ABFD0021302052
:1021C000FFF7A7FD00218D20FFF7A3FD00211420BC
:1021D000FFF79FFD0021AF20FFF79BFD08BD00002A
:1021E00029000020000C014008B501210C2000F05E
:1021F00079FD3C20ADF8000001208DF80200482058
:102200008DF8030069468C4800F0B0FA40F60340B0
:10221000ADF8000010208DF8030003208DF80200B7
:102220006946864800F0A2FA08BD70B51025002066
:102230008349086001208349C1F880018049243125
:1022400008608049C1F8AC017B4800F02BFB0446D4
:1022500004F03C043C2C2AD0142000F032F97648DB
:1022600000F020FB044604F03C043C2C1FD07248D4
:1022700000F018FB00F03C041C2C0BD02C2C07D0D9
:10228000342C03D0382C07D10C2506E00D2504E0B2
:102290000E2502E00F2500E000BF00BF05E0664804
:1022A00000F000FB044604F03C043C2CF7D1012074
:1022B0006349086000206349C1F88001012060493A
:1022C000243108605F49C1F8AC015B4800F0EAFACC
:1022D000044604F03C043C2C2AD0142000F0F1F811
:1022E000554800F0DFFA044604F03C043C2C1FD0B3
:1022F000514800F0D7FA00F03C041C2C0BD02C2CD9
:1023000007D0342C03D0382C07D1032506E006254E
:1023100004E0092502E00B2500E000BF00BF05E056
:10232000454800F0BFFA044604F03C043C2CF7D1C9
:102330000120434908604349C1F880010020404919
:102340002431086001203F49C1F8AC013A4800F04F
:10235000A9FA044604F03C043C2C2AD0142000F0D6
:10236000B0F8354800F09EFA044604F03C043C2CDA
:102370001FD0314800F096FA00F03C041C2C0BD022
:102380002C2C07D0342C03D0382C07D1012506E0A3
:10239000042504E0072502E00A2500E000BF00BF95
:1023A00005E0254800F07EFA044604F03C043C2C8D
:1023B000F7D10120224908602249C1F88001204953
:1023C0002431086000201F49C1F8AC011A4800F010
:1023D00069FA044604F03C043C2C2AD0142000F096
:1023E00070F8154800F05EFA044604F03C043C2CFA
:1023F0001FD0114800F056FA00F03C041C2C0BD002
:102400002C2C07D0342C03D0382C07D1022506E021
:10241000052504E0082502E0002500E000BF00BF1C
:1024200005E0054800F03EFA044604F03C043C2C6C
:10243000F7D1284670BD000000080140000C0140A3
:10244000848121420080214210B56FF0040000F029
:1024500000FF2E4800682E49B0FBF1F02D490870AE
:102460000846007800EB4001C1EBC0104FF6FF7149
:1024700001EAC0002849088010BD0146254A1278AB
:102480004A434FF0E0235A6100229A611A461269CA
:1024900042F001021A6100BF4FF0E022106900F023
:1024A00001021AB100F48032002AF5D04FF0E02288
:1024B000126922F001024FF0E0231A6100229A61B2
:1024C00070470146144A12884A434FF0E0235A618C
:1024D00000229A611A46126942F001021A6100BF95
:1024E0004FF0E022106900F001021AB100F48032CE
:1024F000002AF5D04FF0E022126922F001024FF0DD
:10250000E0231A6100229A61704700001400002045
:1025100000127A006A0100206C010020014600BF11
:10252000704700BF544A128802F04002002AF9D0D6
:10253000C2B2514B1B1D1A80704770B505460E463E
:10254000002400BF0BE000BF40214B4800F0D8FD45
:102550000028F9D0295D484800F064FD641CB442AD
:10256000F1DB70BD10B586B00446012144F20400D1
:1025700000F0B8FB4FF40070ADF8140003208DF8A4
:10258000160018208DF8170005A93C4800F0EEF859
:102590004FF48060ADF8140004208DF8170005A9F1
:1025A000364800F0E3F825208DF8000003208DF870
:1025B00001008DF8020001208DF80300684600F04C
:1025C000FEFD01940020ADF80800ADF80A00ADF85A
:1025D0000C00ADF810000C20ADF80E0001A9264843
:1025E00000F027FC012240F22551234800F0B9FCFD
:1025F0000121214800F0A9FC06B010BD10B540F241
:1026000025511D4800F092FD10B31B4800F00EFD4F
:10261000C4B21B48008800F40040C8B918480088BC
:1026200000F4804060B10A2C03D0002014490880D7
:1026300020E01348008840F400401149088019E068
:102640000D2C06D10E48008840F480400C490880CB
:1026500010E00B480088C0F30D000A490C540848EC
:102660000088401C0649088008460088C72801DD0C
:102670000020088010BD0000003801400008014023
:102680007401002080020020064880470648004769
:10269000FEE7FEE7FEE7FEE7FEE7FEE7FEE7FEE712
:1026A000FEE7FEE763100008ED00000810B50446E1
:1026B000CC48844208D10121042000F02DFB0021E8
:1026C000042000F029FB46E0C748844208D10121DC
:1026D000082000F021FB0021082000F01DFB3AE05B
:1026E000C248844208D10121102000F015FB0021CE
:1026F000102000F011FB2EE0BD48844208D10121DA
:10270000202000F009FB0021202000F005FB22E042
:10271000B848844208D10121402000F0FDFA002190
:10272000402000F0F9FA16E0B348844208D10121B4
:10273000802000F0F1FA0021802000F0EDFA0AE09C
:10274000AE48844207D10121801500F0E5FA00214E
:10275000A01500F0E1FA10BD10B50121084600F007
:10276000DBFA0021012000F0D7FA10BD2DE9F0417D
:10277000024600250026002000230024002791F8AF
:1027800003C00CF00F0591F803C00CF0100CBCF165
:10279000000F03D091F802C04CEA050591F800C083
:1027A000BCF1000F31D0146800202BE04FF0010C79
:1027B0000CFA00F3B1F800C00CEA03069E4220D1E7
:1027C00083004FF00F0C0CFA03F7BC4305FA03FC2F
:1027D0004CEA040491F803C0BCF1280F06D14FF075
:1027E000010C0CFA00FCC2F814C00AE091F803C016
:1027F000BCF1480F05D14FF0010C0CFA00FCC2F8F7
:1028000010C0401C0828D1D31460B1F800C0BCF13E
:10281000FF0F34DD546800202EE000F1080C4FF06B
:10282000010808FA0CF3B1F800C00CEA03069E4256
:1028300021D183004FF00F0C0CFA03F7BC4305FACB
:1028400003FC4CEA040491F803C0BCF1280F05D145
:1028500000F1080C08FA0CF8C2F8148091F803C0D3
:10286000BCF1480F07D100F1080C4FF0010808FA3D
:102870000CF8C2F81080401C0828CED35460BDE884
:10288000F0814FF6FF710180022181700421C17037
:1028900070470246002093680B400BB1012000E016
:1028A000002070470146886880B2704702460020C9
:1028B000D3680B400BB1012000E0002070470146B7
:1028C000C86880B2704701617047416170470AB1C2
:1028D000016100E041617047C16070474FF4803290
:1028E0000A4382618161826182698269704702461E
:1028F0000020434B18684FF68073184040EA0210DE
:1029000008433F4B186070473E49C8617047F0B5B7
:102910000A46002300240021002500F00046B6F1FD
:10292000004F02D1364EF16901E0354E7168C0F3B7
:10293000034583B200F44016B6F5401F08D121F0DC
:1029400070612F4E766826F070662D4F7E6012E023
:1029500000F48016B6F5801F06D1032606FA05F4AA
:10296000A14341F0706106E0460D360103FA06F618
:10297000B14341F0706122B1460D360103FA06F60B
:10298000314300F00046B6F1004F02D11C4EF16118
:1029900001E01B4E7160F0BD30B500228B071C0FAB
:1029A0000F2303FA04F2164B08338C1053F824302B
:1029B0009343134C08348D1044F8253023468C1073
:1029C00053F824308C07240F00FA04F423430C4CF2
:1029D00008348D1044F8253030BD0A49DC310860D8
:1029E0007047000000080140000C01400010014049
:1029F0000014014000180140001C0140002001406B
:102A00000000014000002042DF48006840F0010063
:102A1000DD49086008464068DC490840DA494860FA
:102A200008460068DA490840D74908600846006847
:102A300020F4802008600846406820F4FE004860CA
:102A40004FF41F0088607047CF49096821F4803136
:102A5000CD4A11601146096821F480211160B0F55A
:102A6000803F03D0B0F5802F0ED106E0C64909683B
:102A700041F48031C44A116007E0C349096841F458
:102A8000A021C14A116000E000BF00BF704710B52F
:102A900001460022002300204A11012A02D1BA4C2B
:102AA000236806E0022A02D1B74C236A01E0B64C43
:102AB000636A01F01F02012494401C400CB1012004
:102AC00000E0002010BD38B5002000900024002553
:102AD00000BF3120FFF7DBFF05460098401C009047
:102AE0000098B0F5A06F01D0002DF2D03120FFF793
:102AF000CEFF08B1012400E00024204638BD014685
:102B00000020A14A106820F0F80040EAC1001060DF
:102B10007047A04908607047024600209A4B5868E9
:102B200020F47C1042EA01031843974B5860704729
:102B300098490866704701460020934A506820F083
:102B400003000843506070478F48406800F00C0055
:102B50007047014600208C4A506820F0F00008437E
:102B60005060704701460020874A506820F4E060BA
:102B700008435060704701460020834A506820F4A3
:102B8000605040EAC1005060704729B17E4A527AD5
:102B900002437D4B5A7204E07B4A527A82437A4B5D
:102BA0005A7270477B49D83108607047014600204F
:102BB000754A506820F44040084350607047002137
:102BC000714A20321170704A82F82010012802D018
:102BD00004280AD104E001216B4A2032117005E07B
:102BE0000521694A2032117000E000BF00BF704724
:102BF0006949086070476449096A0143624A116281
:102C00007047654944390860704730B5002100229B
:102C1000002400235C4D6D6805F00C0121B10429EE
:102C200005D0082923D105E05C4D056022E05B4D0D
:102C300005601FE0544D6D6805F47012524D6D68CB
:102C400005F48034022505EB92421CB9544D5543DE
:102C500005600BE04C4D6D6805F400351DB1504D1D
:102C60005543056002E04D4D5543056002E04B4D74
:102C7000056000BF00BF444D6D6805F0F001090913
:102C8000484D6B5C0568DD4045603F4D6D6805F45F
:102C9000E061090A434D6B5C4568DD4085603A4D53
:102CA0006D6805F46051C90A3E4D6B5C4568DD40B6
:102CB000C560354D6D6805F44041890B3A4D6B5C3C
:102CC000C568B5FBF3F5056130BD29B12E4A5269DF
:102CD00002432D4B5A6104E02B4A526982432A4B2E
:102CE0005A61704729B1284A92690243264B9A617A
:102CF00004E0254A92698243234B9A61704729B1C7
:102D0000214AD2690243204BDA6104E01E4AD269AB
:102D100082431D4BDA61704729B11B4AD2680243D6
:102D2000194BDA6004E0184AD2688243164BDA6025
:102D3000704729B1144A12690243134B1A6104E027
:102D4000114A12698243104B1A6170471249403987
:102D5000086070470F49C86470470B49C8717047D5
:102D60000948406A40F08070074948627047014650
:102D70000020054A92680A400AB1012000E00020C4
:102D80007047014988727047001002400000FFF848
:102D9000FFFFF6FE000042428004424200127A0029
:102DA00000093D00760100208601002010B5044690
:102DB000FB48844209D101218803FFF7ADFF0021C0
:102DC0004FF48040FFF7A8FF32E0F648844209D173
:102DD00001214804FFF7ADFF00214FF40030FFF759
:102DE000A8FF25E0F048844209D101218804FFF7BB
:102DF000A0FF00214FF48020FFF79BFF18E0EB4875
:102E0000844209D10121C804FFF793FF00214FF448
:102E10000020FFF78EFF0BE0E548844208D1012136
:102E20000805FFF786FF00214FF48010FFF781FFB0
:102E300010BD2DE9F04786B005460E460024A24697
:102E400000BFA1460027B08900B100BF2F462C8AE1
:102E50004CF6FF700440F08804432C82AC894EF697
:102E6000F3100440B0883189084371890843044352
:102E7000AC81AC8A4FF6FF400440B0890443AC8279
:102E800001A8FFF7C2FEC648874202D1DDF810A0B4
:102E900001E0DDF80CA0A88900F4004040B10AEB85
:102EA000CA0000EB0A1031684900B0FBF1F807E0F6
:102EB0000AEBCA0000EB0A1031688900B0FBF1F898
:102EC0006420B8FBF0F004012009642101FB1089A3
:102ED000A88900F4004040B1322000EBC900B0FBEB
:102EE000F1F000F00700044308E0322000EB091085
:102EF0006421B0FBF1F000F00F0004432C8106B018
:102F0000BDE8F0874FF41651016000218180C18037
:102F100001810C21418100218181704710B5024659
:102F20000020108A4FF2FF0318400B884C8823437F
:102F30008C882343CC8823431843108210BD002182
:102F4000018041808180C180704721B1828942F433
:102F50000052828104E082894DF6FF731A4082811B
:102F60007047F0B50346002400260025002040F6F7
:102F70006A17B94200D100BF1846C1F3421401F0EC
:102F80001F06012707FA06F5012C01D10C3004E0D9
:102F9000022C01D1103000E014301AB107682F4321
:102FA000076002E00768AF430760F0BD1AB1838A8B
:102FB0000B43838202E0838A8B4383827047028AB9
:102FC0004FF6F0731A400282028A0A430282704767
:102FD00082894FF2FF731A40828182890A4382817B
:102FE000704721B1828942F00202828104E0828925
:102FF0004FF6FD731A4082817047028A4FF6DF73E5
:103000001A400282028A0A430282704721B1028A70
:1030100042F48042028204E0028A4BF6FF731A40B7
:1030200002827047C1F30802828070470146888897
:10303000C0F308007047818941F001018181704728
:10304000028BD2B20283028B42EA012202837047D2
:10305000028B02F47F420283028B0A430283704791
:1030600021B1828A42F02002828204E0828A4FF6F5
:10307000DF731A408282704721B1828A42F01002C7
:10308000828204E0828A4FF6EF731A408282704790
:1030900021B1828A42F00802828204E0828A4FF6DD
:1030A000F7731A408282704721B1828942F400424C
:1030B000828103E08289C2F30E028281704721B1CE
:1030C000828A42F40062828204E0828A4FF2FF73B5
:1030D0001A4082827047828A4FF6FB731A408282BE
:1030E000828A0A438282704721B1828A42F00202B8
:1030F000828204E0828A4FF6FD731A408282704712
:1031000002460020B1F5007F00D100BF13880B40BC
:103110000BB1012000E00020704701F40072B2F50D
:10312000007F00D100BFCA430280704770B50246DD
:10313000002400230025002040F66A16B14200D189
:1031400000BFC1F3421501F01F03012606FA03F385
:10315000012D02D19689334006E0022D02D1168A54
:10316000334001E0968A33400C12012606FA04F43B
:103170001688344013B10CB1012000E0002070BD6E
:1031800010B50022002340F66A14A14200D100BF0E
:103190000A1201249440A3B2DC43048010BD000055
:1031A000003801400044004000480040004C00400E
:1031B0000050004031490143314A1160704770B5F9
:1031C000002100230F22C47804B32D4C246804F49A
:1031D000E064C4F5E064210AC1F10403CA40447804
:1031E00004FA03F18478144021430901254C067840
:1031F000A155047804F01F050124AC4005786D1139
:10320000AD0005F1E025C5F8004109E0047804F0BF
:103210001F050124AC401C4D0678761145F8264068
:1032200070BD1A4A0A400243154B1B1F1A607047B3
:1032300039B1134A121D12680243114B1B1D1A604B
:1032400006E00F4A121D126882430D4B1B1D1A60C7
:103250007047042808D14FF0E021096941F00401CA
:103260004FF0E022116107E04FF0E021096921F001
:1032700004014FF0E0221161704700000000FA05E0
:103280000CED00E000E400E080E100E080FFFF1FC3
:1032900010B50446FA48844208D101214015FFF7D1
:1032A0003BFD00216015FFF737FD17E0F54884422C
:1032B00008D101210015FFF72FFD00212015FFF790
:1032C0002BFD0BE0F048844208D10121C803FFF731
:1032D00023FD00214FF40040FFF71EFD10BD30B567
:1032E0000246002000235068E84C20400D790C680D
:1032F00044EA0524204350609068E54C2040D1E921
:1033000002542C434D7944EA450420439060D06A2E
:1033100020F470000C7C641EE4B2234340EA0350A6
:10332000D06230BD00210160017141718160C160D6
:1033300001210174704721B1826842F0010282606C
:1033400003E0826822F001028260704721B1826846
:1033500042F48072826003E0826822F480728260AC
:10336000704710B50023CBB21AB144681C434460C7
:1033700002E044689C43446010BD816841F008014C
:1033800081607047014600208A6802F008020AB195
:10339000012000E000207047816841F00401816055
:1033A0007047014600208A6802F004020AB1012039
:1033B00000E00020704721B1826842F4A0028260E0
:1033C00003E0826822F4A002826070470146002078
:1033D0008A6802F480020AB1012000E000207047F0
:1033E00010B50A4600210023416821F46041531EB4
:1033F00041EA4331416010BD21B1426842F40062AC
:10340000426003E0426822F4006242607047F0B517
:1034100004460D4600200021092D11DDE068A5F1CC
:103420000A0606EB4607072606FA07F18843A5F1C8
:103430000A0606EB460603FA06F10843E0600CE0D4
:10344000206905EB4507072606FA07F1884305EBD7
:10345000450603FA06F108432061072A0FDA606B7C
:10346000561E06EB86071F2606FA07F18843561EEE
:1034700006EB860605FA06F10843606322E00D2A92
:103480000FDA206BD61F06EB86071F2606FA07F118
:103490008843D61F06EB860605FA06F1084320632B
:1034A00010E0E06AA2F10D0606EB86071F2606FA79
:1034B00007F18843A2F10D0606EB860605FA06F130
:1034C0000843E062F0BD21B1826842F4801282605C
:1034D00003E0826822F48012826070470146C86C63
:1034E00080B2704766484C300068704721B142682E
:1034F00042F48062426003E0426822F480624260EB
:10350000704721B1426842F48052426003E0426851
:1035100022F48052426070470A460021816821F4FB
:10352000E04111438160704721B1826842F400425A
:10353000826003E0826822F400428260704721B119
:10354000826842F40212826003E0826822F402126E
:1035500082607047014600208A6802F400120AB1B6
:10356000012000E000207047F0B504461546002019
:1035700000220026092911DDE068A1F10A0707EB06
:10358000470C072707FA0CF29043A1F10A0707EB53
:10359000470703FA07F21043E0600CE0206901EBF3
:1035A000410C072707FA0CF2904301EB410703FA9D
:1035B00007F210432061A06BC0F30156EF1C06F127
:1035C000010CA7EB0C0707EB870C1F2707FA0CF27F
:1035D0009043EF1C06F1010CA7EB0C0707EB8707E4
:1035E00001FA07F21043A063F0BD10B50A460021AE
:1035F0000023816B21F44011531E41EA0351816382
:1036000010BD08B5002300930090009B0B4400936D
:10361000009B1A6008BD08B5024600200090009289
:1036200001F12800009B184400900098006880B2C7
:1036300008BD0A4600214168164B194011434160FC
:1036400070474162826270470A460021416821F05A
:103650001F0111434160704740B1094908310968B1
:1036600041F40001064A0832116007E004490831BC
:10367000096821F40001024A083211607047000015
:103680000024014000280140003C0140FFFEF0FF03
:10369000FDF7F1FFFFFD3FFF0246002013680B40DE
:1036A0000BB1012000E000207047CA430260704760
:1036B00070B502460020002300240B125568CEB2DC
:1036C00005EA060415681D4015B10CB1012000E0A3
:1036D000002070BD00220A12D3430360704700002F
:1036E00010B50446FE48844208D10121C014FFF7FA
:1036F00013FB0021E014FFF70FFBC4E0B4F1804F8F
:1037000008D101210846FFF714FB00210120FFF733
:1037100010FBB8E0F348844208D101210220FFF7F2
:1037200008FB00210220FFF704FBACE0EE488442D6
:1037300008D101210420FFF7FCFA00210420FFF743
:10374000F8FAA0E0E948844208D101210820FFF7F7
:10375000F0FA00210820FFF7ECFA94E0E4488442F4
:1037600008D101211020FFF7E4FA00211020FFF713
:10377000E0FA88E0DF48844208D101212020FFF7E9
:10378000D8FA00212020FFF7D4FA7CE0DA488442FE
:1037900008D101214014FFF7BFFA00216014FFF7A0
:1037A000BBFA70E0D548844209D10121C804FFF773
:1037B000B3FA00214FF40020FFF7AEFA63E0D048DF
:1037C000844209D101210805FFF7A6FA00214FF430
:1037D0008010FFF7A1FA56E0CA48844209D10121BE
:1037E0004805FFF799FA00214FF40010FFF794FA0B
:1037F00049E0C548844208D101214020FFF799FAE9
:1038000000214020FFF795FA3DE0C048844208D1EE
:1038100001218020FFF78DFA00218020FFF789FA2F
:1038200031E0BB48844208D101218015FFF781FABD
:103830000021A015FFF77DFA25E0B648844209D1A2
:1038400001210804FFF768FA00214FF48030FFF7E8
:1038500063FA18E0B048844209D101214804FFF717
:103860005BFA00214FF40030FFF756FA0BE0AB484B
:10387000844208D101218804FFF74EFA00214FF459
:103880008020FFF749FA10BD00220288944B98422D
:103890000ED0994B98420BD0B0F1804F08D0914B8D
:1038A000984205D0904B984202D0904B984204D158
:1038B0004FF68F731A404B881A438D4B984207D0AE
:1038C0008C4B984204D04FF6FF431A40CB881A43E2
:1038D00002808B8883850B880385814B98420BD0AF
:1038E000854B984208D08B4B984205D08A4B984222
:1038F00002D08A4B984201D10B7A0386012383823E
:10390000704770B5002400220023058C4FF6FE7628
:1039100035400584028C8388048B4FF68F752C40CC
:10392000B51E2C400D882C43751E2A400D892A4354
:103930004D882A436A4DA8420BD06F4DA84208D04B
:10394000744DA84205D0744DA84202D0734DA842D0
:1039500013D14FF6F7752A404D892A434FF6FB7570
:103960002A408D882A434FF6FF652B404FF6FF55BE
:103970002B408D892B43CD892B4383800483CD88B5
:103980008586028470BD70B5002400220023058C5A
:103990004FF6EF7635400584028C8388048B48F619
:1039A000FF752C404FF6FF452C400D884FF6FF76F3
:1039B00006EA05252C434FF6DF752A400D8906EAF5
:1039C00005152A434D8806EA05152A43444DA842A9
:1039D00002D0494DA8421DD14FF67F752A404D892E
:1039E0004FF6FF7606EA05152A434FF6BF752A40C3
:1039F0008D8806EA05152A434FF6FF352B404FF216
:103A0000FF752B408D8906EA85052B43CD8906EA93
:103A100085052B4383800483CD880587028470BD90
:103A200070B5002400220023058C4FF6FF66354058
:103A30000584028C8388848B4FF68F752C404FF65B
:103A4000FC752C400D882C434FF6FF552A400D89FC
:103A50004FF6FF7606EA05252A434D8806EA052536
:103A60002A431F4DA84202D0234DA8421DD14FF238
:103A7000FF752A404D894FF6FF7606EA05252A4351
:103A80004FF6FF352A408D8806EA05252A434EF673
:103A9000FF752B404DF6FF752B408D8906EA051505
:103AA0002B43CD8906EA05152B4383808483CD887B
:103AB0008587028470BD70B5002200230024058C28
:103AC0004EF6FF7635400584038C8488828B48F659
:103AD000FF752A404FF6FF452A400D8820E0000080
:103AE000002C01400004004000080040000C004091
:103AF000001000400014004000340140004C014020
:103B0000005001400054014000180040001C0040DB
:103B100000200040004001400044014000480140B6
:103B20004FF6FF7606EA05252A434DF6FF752B4032
:103B30000D8906EA05352B434D8806EA05352B43EA
:103B4000FA4DA84202D0FA4DA84208D14BF6FF75B3
:103B50002C408D894FF6FF7606EA85152C4384802C
:103B60008283CD88A0F84050038470BD828B4FF2D1
:103B7000FF331A408283828B4FF6FF7303EA0123DF
:103B80001A4382837047F0B50C4615460022002187
:103B90000026078C4EF6FF7C07EA0C070784828B11
:103BA000018C4FF6FF7707EA043640F6FF473A40AC
:103BB0004FF6FF7707EA05273A434FF6FF7707EA04
:103BC00003373A43D94FB8420ED0D94FB8420BD041
:103BD000B0F1804F08D0D74FB84205D0D64FB84289
:103BE00002D0D64FB84206D14DF6FF77394046F4A1
:103BF0008057394305E047F6FF57394044F4805772
:103C0000394382830184F0BD828B4FF6F3731A40EF
:103C10008283828B0A4382837047F0B50C46154637
:103C2000002200210026078C4FF6FF6C07EA0C07E4
:103C30000784828B018C4FF6FF7707EA04264FF644
:103C40000C773A404FF6FF7707EA03172F433A43C2
:103C5000B64FB8420ED0B64FB8420BD0B0F1804F3D
:103C600008D0B44FB84205D0B34FB84202D0B34FDA
:103C7000B84206D14FF6FF57394046F480773943B2
:103C800005E04FF2FF57394044F48077394382838F
:103C90000184F0BD028B4FF2FF331A400283028B86
:103CA0004FF6FF7303EA01231A4302837047F0B50E
:103CB0000C461546002200210026078C4FF6EF7CAB
:103CC00007EA0C070784028B018C4FF6FF7707EA9F
:103CD000041640F6FF473A404FF6FF7707EA0337EE
:103CE0003A434FF6FF7707EA05273A438F4FB8422A
:103CF0000ED08F4FB8420BD0B0F1804F08D08D4F0F
:103D0000B84205D08C4FB84202D08C4FB84206D191
:103D10004FF6DF77394046F01007394305E04FF69C
:103D20005F77394044F01007394302830184F0BDC6
:103D3000028B4FF6F3731A400283028B0A4302830D
:103D40007047F0B50C46154600220021068C4FF650
:103D5000FE773E400684028B018C4FF60C76324093
:103D60007E1C06EA03162E433243704EB0420ED03C
:103D70006F4EB0420BD0B0F1804F08D06D4EB042C4
:103D800005D06D4EB04202D06C4EB04206D14FF617
:103D9000FD76314044F00106314305E04FF6F576FB
:103DA000314044F00106314302830184F0BD70B517
:103DB00005460C465D4885420ED05D4885420BD0D5
:103DC000B5F1804F08D05B48854205D05A488542FE
:103DD00002D05A48854200D100E000BF208850B987
:103DE0002389A28861882846FFF7ABFFE18828462F
:103DF000FFF79EFF25E0208804280AD12389A288A6
:103E000061882846FFF753FFE1882846FFF742FF05
:103E100017E0208808280AD12389A28861882846CB
:103E2000FFF7FBFEE1882846FFF7EEFE09E0238955
:103E3000A28861882846FFF7A6FEE1882846FFF79A
:103E400095FE70BD2DE9F04105460C460026012780
:103E5000608808B9022600E00026A088012801D168
:103E6000022700E001272088A0B92389A288618861
:103E70002846FFF766FFE1882846FFF759FF2389A8
:103E80003A4631462846FFF712FFE1882846FFF7F9
:103E900001FF13E02389A28861882846FFF707FF06
:103EA000E1882846FFF7F6FE23893A463146284640
:103EB000FFF747FFE1882846FFF73AFFBDE8F081AA
:103EC0000A884B881A438B881A43CB881A430B897C
:103ED0001A434B891A438B891A43A0F84420704730
:103EE0004FF6FF71818000210180C1804180017205
:103EF00070470021018041808180C1800181418122
:103F00008181C18170470021018041800121818030
:103F10000021C180018170470021018041808180A2
:103F2000C18001814181818170470000002C0140E6
:103F3000003401400004004000080040000C004034
:103F400021B1028842F00102028004E002884FF6AB
:103F5000FE731A400280704731B1B0F8442042F439
:103F60000042A0F8442005E0B0F84420C2F30E025D
:103F7000A0F8442070471AB183890B43838102E083
:103F800083898B43838170478182704741EA0203B2
:103F9000A0F8483070471AB183890B43838102E04F
:103FA00083898B438381704701894FF6F8721140F2
:103FB000018170470A46002101894FF68F7319402D
:103FC00011430181704730B504460D46294620460D
:103FD000FFF7F0FF208940F00700208130BD2DE978
:103FE000F04104460D4616461F46602D06D13B465D
:103FF000012231462046FFF75AFE05E03B460122EA
:1040000031462046FFF79DFE29462046FFF7D2FFA6
:10401000208940F007002081BDE8F08130B50C46D2
:1040200000210189C9B24FF6FF7505EA0325154342
:1040300025432943018130BD2DE9F04105460E4657
:1040400017469846002443463A4631462846FFF72D
:10405000E5FF2C894FF6F870044044F007044FF652
:104060008F70044044F070042C81BDE8F081F0B5FD
:1040700004460D4616461F463B4632462946204614
:10408000FFF7CCFF208940F480402081F0BD0185FE
:10409000828270470A46002101884FF68F731940CB
:1040A000114301807047F0B50C4615461E460021AD
:1040B000002200230189028B038C4FF6F8773940E8
:1040C00021434FF6FC473A4040F201173A434FF67E
:1040D000DD773B404FF6FF7707EA06172F433B4358
:1040E000018102830384F0BD0A460021018B4FF653
:1040F0008F7319401143018370470A460021018BD9
:1041000048F6FF7319404FF6FF7303EA0223194381
:10411000018370470A460021818B4FF68F73194047
:104120001143818370470A460021818B48F6FF7353
:1041300019404FF6FF7303EA022319438183704746
:1041400021B1028842F08002028004E002884FF62A
:104150007F731A400280704721B1828842F00402C6
:10416000828004E082884FF6FB731A408280704799
:1041700021B1828842F00802828004E082884FF6F2
:10418000F7731A408280704721B1828842F00102A1
:10419000828004E082884FF6FE731A408280704766
:1041A0000A460021018B4FF6F77319401143018332
:1041B00070470A460021018B4FF2FF7319404FF6FA
:1041C000FF7303EA02231943018370470A46002163
:1041D000818B4FF6F77319401143818370470A466C
:1041E0000021818B4FF2FF7319404FF6FF7303EAF2
:1041F00002231943818370470A460021018B4FF641
:10420000FB7319401143018370470A460021018B5B
:104210004FF6FF3319404FF6FF7303EA02231943A9
:10422000018370470A460021818B4FF6FB731940CA
:104230001143818370470A460021818B4FF6FF337B
:1042400019404FF6FF7303EA022319438183704735
:104250000A460021018B4FF67F73194011430183F9
:1042600070470A460021018BC1F30E014FF6FF7320
:1042700003EA02231943018370470A460021818B18
:104280004FF67F7319401143818370470A4600211E
:10429000818BC1F30E014FF6FF7303EA022319432A
:1042A000818370470A460021018C4FF6FD73194047
:1042B0001143018470470A460021018C4FF6F773C1
:1042C00019401143018470470A460021018C4FF6C2
:1042D000DF7319404FF6FF7303EA02131943018499
:1042E00070470A460021018C4FF67F7319404FF644
:1042F000FF7303EA02131943018470470A46002141
:10430000018C4FF6FF5319404FF6FF7303EA022367
:104310001943018470470A460021018C4FF2FF7354
:1043200019404FF6FF7303EA0223194301847047D3
:104330000A460021018C4DF6FF7319404FF6FF73BA
:1043400003EA023319430184704730B50023012486
:104350008C40A3B2048C9C430484048C02FA01F5C3
:10436000ADB22C43048430BD30B5002304248C400E
:10437000A3B2048C9C430484048C02FA01F5ADB210
:104380002C43048430BD70B5034600200024184639
:10439000183001258D40ACB21D8CA5431D8409B198
:1043A000082909D100EB6100056825F0700505605A
:1043B0000568154305600EE00D1FC5F34E05284442
:1043C000056825F4E045056005684FF6FF7606EAC6
:1043D00002263543056070BD21B1028842F0020219
:1043E000028004E002884FF6FD731A400280704795
:1043F00021B1028842F00402028004E002884FF6F4
:10440000FB731A400280704721B1828842F080021B
:10441000828004E082884FF67F731A408280704762
:1044200002884FF6F7731A40028002880A4302801E
:10443000704782884FF68F731A40828082880A43C1
:104440008280704702894FF6F8731A400281028910
:104450000A430281704702894FF67F731A40028136
:1044600002890A43028170478184704781857047C1
:10447000818670470187704781877047A0F8401098
:10448000704702884FF6FF431A40028002880A43B1
:10449000028070470146888E70470146088F70473A
:1044A0000146888F70470146B1F8400070470146C9
:1044B000888C70470146088D704702460020138A99
:1044C0000B400BB1012000E000207047CA4302827C
:1044D000704730B50246002000230024158A05EA03
:1044E0000103958905EA010413B10CB1012000E034
:1044F000002030BDCA430282704740EA01039B0797
:1045000003D009E008C9121F08C0042AFAD203E048
:1045100011F8013B00F8013B521EF9D27047D2B2AC
:1045200001E000F8012B491EFBD270470022F6E79C
:1045300010B513460A4604461946FFF7F0FF204619
:1045400010BD30B505462A460B4612F8010B13F88C
:10455000014B08B1A042F8D01CB1002802D06D1C5C
:10456000F1E7284630BDF0B480EA0102D40F4200E2
:10457000B2EB410F02D20246084611464A0042D031
:10458000C30DDDB2C1F3C752AD1A202D35DAC1F328
:10459000160141F4000204B15242C5F1200602FAAC
:1045A00006F12A411044B3EBD05F23D0C4B1012DF2
:1045B000A0EBC35009DCF0BC4FF0004202EAC3524A
:1045C000DBB200F5000000F099B9400000F1807006
:1045D00000EBC350A0F1807040EAD170490009E0BF
:1045E000490841EAC071A0EBC35000F50000400843
:1045F00000EBC350F0BC00F078B96142012202EB3D
:104600004101001BF6E7F0BC704781F00041AAE7CA
:1046100080F00040A7E72DE9FE4F81EA030404F093
:10462000004421F0004100944FF0000B23F00043C0
:1046300050EA01045ED052EA03045BD0C3F30A548B
:10464000C1F30A552C44A4F2F3340194A0FB0254A4
:10465000C1F3130141F48011C3F3130343F4801336
:1046600001FB024400FB034E840A970A44EA81548A
:1046700047EA8357A4FB076802958D0A05FB078567
:104680004FEA932C04FB0C542705029D4FEA065871
:1046900047EA1637B5EB08056EEB070C870E920E4E
:1046A00047EA811742EA8312A7FB0201B6EB0B012E
:1046B00064EB00042B0D43EA0C335E1844EB1C50F2
:1046C000DA465146E7FB0201C5F313044FEA0B3308
:1046D00043EA14534FEA0432019C43EA0603A4F16F
:1046E0000C040294009CCDE900B400F044F903B03E
:1046F000BDE8F08F00200146F9E7C10F80EAE070C5
:104700000844CA079623002100F0F8B89623002237
:10471000114600F0F3B870B5C1F30A5201F000453C
:104720000024C1F3130140F2FF3341F480119A4297
:1047300001DA002070BD40F233439A42A2F23342C4
:1047400003DC524200F0C1F800E090402C43F1D06D
:10475000404270BD00F0004230F000400AD0C10D70
:1047600001F56071C0F3160042EA0151C20840072A
:1047700011437047002001467047000030B5041E09
:1047800071F1000404DB4FF00044404264EB01018E
:10479000141E73F1000405DB1C464FF00043524227
:1047A00063EB04038B4208BF824230BD30B5041E68
:1047B00071F1000404DB4FF00044404264EB01015E
:1047C000141E73F1000405DB1C464FF000435242F7
:1047D00063EB0403994208BF904230BD01F00043EF
:1047E00030B421F0004150EA010206D00A0DA2F5D2
:1047F0006072C1F31301002A02DC30BC0020704754
:10480000440F44EAC104C100E01830BC00EBC250C0
:1048100000F06BB8002801DBC0F10040002901DB8B
:10482000C1F1004181427047002801DBC0F1004026
:10483000002901DBC1F100418842704730B50B46C9
:10484000014600202022012409E021FA02F59D42C0
:1048500005D303FA02F5491B04FA02F52844151E94
:10486000A2F10102F1DC30BD2DE9F05F0546002028
:1048700092469B4688460646814640241BE02846D1
:1048800041464746224600F020F853465A46C01A91
:10489000914110D311461846224600F0FBF92D1A1B
:1048A00067EB01084F4622460120002100F0F2F993
:1048B00017EB00094E41201EA4F10104DFDC48463D
:1048C00031462A464346BDE8F09F202A04DB203AC1
:1048D00021FA02F00021704721FA02F3D040C2F120
:1048E000200291400843194670470029A8BF70472D
:1048F000401C490008BF20F00100704710B4B0FA16
:1049000080FC00FA0CF050EA010404BF10BC7047B0
:1049100049B1CCF1200421FA04F411FA0CF118BFCA
:10492000012121430843A3EB0C01CB1D4FEA006199
:104930004FEA102042BF002010BC704700EBC3506C
:1049400010440029A4BF10BC7047401C490008BF98
:1049500020F0010010BC704710B5141E73F1000464
:1049600008DA401C41F1000192185B411A4301D161
:1049700020F0010010BD2DE9F04D92469B4611B18B
:10498000B1FA81F202E0B0FA80F22032904600F0F3
:1049900081F904460F4640EA0A0041EA0B015346FA
:1049A0005A46084313D0114653EA010019D0C8F102
:1049B00040025046FFF789FF05460E4650465946CD
:1049C000424600F067F9084305D0012004E0204684
:1049D0003946BDE8F08D0020054346EAE0762C43D9
:1049E00037430A986305E40AA0EB08000022FD0A99
:1049F00044EA47540A3002D500200146E9E70105A0
:104A000010196941DDE9084500196941BDE8F04D1B
:104A1000A2E72DE9FE4F804681EA0300C00F0C4655
:104A2000009021F0004123F00045B8EB0200A941BD
:104A300005D24046214690461C460B46024623F0CE
:104A40000040104347D0270DC7F30A00C3F30A51B3
:104A50000290401A019040286BDAC3F3130040F42F
:104A6000801B0098924620B10023D2EB030A63EB2F
:104A70000B0B01985946C0F14002504600F00AF96C
:104A800006460D4650465946019A00F012F910EBC1
:104A900008006141002487EA115284EAE7731A434F
:104AA00040D0009A62B3019A012A4FEA075215DCFE
:104AB000001B61EB02014FF0004202EA0752CDE910
:104AC0000042001C41F5801132462B46FFF753FF90
:104AD00003B0BDE8F08F40462146F9E7001B61EBCB
:104AE0000201001C41F5801300185B412018A2F55B
:104AF000001747EB030140EAD570B6196D4111E08C
:104B00006D084FEA360645EAC0754FEA0752001BAA
:104B100061EB0201001C41F5801149084FEA3000A9
:104B20000019514132462B4603B0BDE8F04FFFF764
:104B300013BF0098012240000023D0EB020263EB78
:104B4000E073009821464FEAE074B8EB000061EB97
:104B50000401E9E783F000435BE781F0004158E797
:104B60002DE9F04D81EA030404F0004B21F00045EB
:104B700014464FF0000A23F0004150EA050220D00D
:104B800054EA01021DD0C5F30A570246C5F31303C8
:104B9000C1F31300C1F30A5640F4801543F48013A7
:104BA000A7EB0608101BD64608F2FD3873EB05008C
:104BB00002D308F1010801E092185B41B8F1000F3F
:104BC00003DA00200146BDE8F08D00204FF480118B
:104BD000064684460EE0171B73EB050705D3121B30
:104BE00063EB050306434CEA010C49084FEA300029
:104BF00092185B4150EA0107EDD152EA030012D04E
:104C000082EA040083EA0501084305D0101BAB418A
:104C100006D20122002306E000224FF0004302E00A
:104C20006FF0010253101AEB06004CEB085110EB29
:104C30000A0041EB0B01BDE8F04DFFF78DBEC1F35B
:104C40000A52C1F3130140F2FF3341F480119A423A
:104C500002DA00200146704740F233439A42A2F242
:104C6000334202DC5242FFF730BE00F013B80000BE
:104C7000064C074D06E0E06840F0010394E80700A9
:104C800098471034AC42F6D3FBF734FAB05E000814
:104C9000D05E0008202A04DB203A00FA02F100204E
:104CA00070479140C2F1200320FA03F3194390406A
:104CB0007047202A06DBCB17203A41FA02F043EA7C
:104CC000E07306E041FA02F3D040C2F120029140C5
:104CD00008431946704730B58C1810F8012B12F0B4
:104CE0000F0301D110F8013B120906D110F8012B76
:104CF00003E010F8015B01F8015B5B1EF9D101E0F4
:104D000001F8013B521EFBD1A142E6D3002030BD89
:104D10000FB4054B10B503A9044A029800F0EEF851
:104D200010BC5DF814FB0000232500087001002072
:104D30000FB4084B10B504A902AA039800F0DEF8DE
:104D4000044602A9002000F070FC204610BC5DF86B
:104D500014FB00002B56000802E008C8121F08C10F
:104D6000002AFAD170477047002001E001C1121FEC
:104D7000002AFBD1704700002DE9FF5F82B00021BF
:104D8000DDE90430020DDDF840B0034318D044F6ED
:104D90001050A2F2FF3242431514119801281FD07F
:104DA000A5EB0B00401C5FEA000A4FF000064E4FD7
:104DB000DFF83891B046504615D5CAF1000413E02B
:104DC000119801244AA3012801D16FEA0B0102982E
:104DD000119AC0E90031C0E9024206B0BDE8F09F77
:104DE000CBF10000DFE704460021404A491842EBBE
:104DF0000450CDE9001012E0E00707D032463B46F0
:104E000040464946FFF707FC8046894632463B4606
:104E100010461946FFF7FFFB06460F466410002CAC
:104E2000EAD1DDE90401DDE90023BAF1000F06DA79
:104E3000FFF7F1FB42464B46FFF7EDFB05E0FFF7BE
:104E40008FFE42464B46FFF78BFE04460E4600227D
:104E5000284BFFF7ABFC03D84FF0FF30014607E0CB
:104E60000022254B20463146FFF7D3FDFFF7E7FE32
:104E7000102409E0002C0ADB0A220023FFF7F4FCCF
:104E8000039B30321A55641E50EA0102F2D1641CB1
:104E9000039AC4F111031444119A012A03D0012288
:104EA00008430DD10AE0084304D000204FF0110B55
:104EB000119072E7A3EB0B056D1E0DE05B4504DD61
:104EC0004FF0000205F1010504E003DA4FF00002A3
:104ED000A5F10105002AECD002981199C0E9023130
:104EE000C0E9004579E70000000014400000F03FF1
:104EF000300000000000F0430000E03F2DE9FF4FCC
:104F000095B09B468946064600250FE2252877D1B5
:104F100000242746F84A0121059400E0044316F8CE
:104F2000013F203B01FA03F01042F7D130782A28E4
:104F300011D06FF02F033078A0F13002092A16D873
:104F4000059A44F0020402EB820203EB4202104491
:104F5000761C0590EFE759F8042B0592002A03DA36
:104F6000504244F40054059044F00204761C30781A
:104F70002E2816D116F8010F44F004042A280DD06B
:104F80006FF02F023078A0F13003092B09D807EB1E
:104F9000870302EB4303C718761CF3E759F8047B39
:104FA000761C30786C280FD006DC4C2817D0682887
:104FB0000DD06A2814D104E0742810D07A280FD1BB
:104FC0000DE044F400140AE044F4801401E044F4D9
:104FD00040147278824202D104F58014761C761C4B
:104FE000307866280BD013DC582877D009DC0028ED
:104FF00075D04528F6D04628F4D047281AD19DE12F
:1050000018E0632835D0642879D0652812D195E15D
:10501000702873D008DC6728F1D069286FD06E281B
:105020000DD06F2806D1B5E073282CD0752875D027
:10503000782874D05A46179990476D1C75E1C4F3CF
:105040000250022809D003280DD0D9F800100428F6
:105050000DD00D6009F1040967E1D9F80010EA17D5
:10506000C1E90052F6E7D9F800100D80F2E70D70A3
:10507000F0E719F8041B8DF8001000208DF80100EE
:10508000EA46012003E059F804AB4FF0FF30610716
:105090004FF0000102D40DE008F101018846B94249
:1050A0000FDA8045F8DB1AF808100029F4D108E07F
:1050B00008F1010188468142FADB1AF8081000293C
:1050C000F6D105985B46A0EB080721463846179AAB
:1050D00000F094FA284400EB080507E04DE029E1D0
:1050E0000DE01AF8010B5A4617999047B8F10108DC
:1050F000F7D25B4621463846179A13E142E00A226E
:105100000092C4F302524FF0000A022A08D059F864
:1051100004CB032A4FEAEC710AD00DE029E02AE023
:1051200009F1070121F00702F2E802C1914609E006
:105130000FFA8CFC4FEAEC71042A03D14FFA8CFC75
:105140004FEAEC71002907DA0A460021DCF1000C75
:1051500061EB02012D2202E0220504D52B228DF8FD
:105160000420012203E0E20701D02022F7E7904665
:1051700059E00A2102E010220DE010214FF0000A50
:1051800000910BE010224FF0000A44F004040827BD
:10519000009203E008224FF0000A0092C4F302528A
:1051A000022A05D059F804CB0021032A08D009E0CF
:1051B00009F1070121F00702F2E802C1914605E07A
:1051C0001FFA8CFC042A01D10CF0FF0C4FF00008F0
:1051D000220728D5702806D0009B83F0100353EADD
:1051E0000A0305D00EE040228DF80420012208E0D9
:1051F0005CEA010206D030228DF804208DF805000B
:1052000002229046009B83F0080353EA0A030AD166
:105210005CEA010201D1620705D530228DF8042035
:105220004FF001087F1E582804D034A003900EA828
:1052300002900DE036A0F9E753466046009AFFF76A
:1052400013FB84460398825C0298401E0290027011
:105250005CEA0100F0D1029806A9081A00F1200AC0
:10526000600702D524F4803400E00127574502DDB1
:10527000A7EB0A0000E0002000EB0A01009005986F
:105280004144401A0590E00306D45B462146179A34
:10529000059800F0B3F90544002706E001A85A4636
:1052A000C05D179990476D1C7F1C4745F6DBE003F6
:1052B0000CD55B462146179A059800F09FF90544E6
:1052C00004E030205A46179990476D1C0099481EFB
:1052D00000900029F5DC08E0029802995A4600780F
:1052E000491C0291179990476D1CBAF10001AAF16F
:1052F000010AF1DC65E10000092801003031323398
:105300003435363738396162636465660000000001
:1053100030313233343536373839414243444546EB
:105320000000000000F058F90544761C3078002891
:105330007FF4ECAD19B02846BDE8F08F620700D4C9
:10534000062709F1070222F0070CFCE80223E146D8
:1053500003F000485FEA080C02D00FF2702C0DE059
:105360005FEA045C02D50FF2682C07E05FEAC47CB8
:1053700002D00FF2602C01E0AFF2700C4FF0FF385A
:1053800023F00043CDF850C065280CD006DC45283A
:1053900009D046281DD047283DD13DE0662818D0C9
:1053A00067287ED138E00021112F01DB112000E0B9
:1053B000781CCDE9000106A90EA8FFF7DDFCDDE9A8
:1053C0000F010E9A03910021009207F1010A049146
:1053D0004DE04FF000400097CDE9011006A90EA85E
:1053E000FFF7CAFCDDE90F0203920E9B1199002220
:1053F000DDF80CA00093049211B9791C00EB010AAE
:10540000B7EB0A0004D4C0F1FF3007F1010A0490A1
:10541000AAEB0700019044E0012F00DA01270021E8
:10542000112F01DD112000E03846CDE9000106A969
:105430000EA8FFF7A1FCDDE90F010E9A03910021F0
:1054400004910092BA4621070CD40399514500DA21
:105450008A46BAF1010F05DD009AAAF10101515CFB
:10546000302908D0B84202DA10F1040F06DA01211F
:10547000CDE9011015E0AAF10101E9E7002805DCFA
:10548000049901440491AAEB000102E0411C51453A
:1054900000DD8A460499401A401C01904FF00040FC
:1054A0000290200704D40198504501DBCDF8048018
:1054B00000208DF84F0002980DF14F07B0F1004F1A
:1054C00025D02B200E9002984FF0020800280CDA0D
:1054D000404202902D200E9007E00A210298FFF72B
:1054E000ADF93031029007F8011DB8F10001A8F1C3
:1054F0000108F2DC02980028EFD1791E0E9808709E
:10550000307800F0200040F0450007F8020D12A8A6
:10551000C01B00F107081498007800B1012000EBCF
:105520000A01019801EBE07105984144401A401EC0
:105530000590E00306D45B462146179A059800F0D3
:105540005DF805441498007818B15A4617999047A9
:105550006D1CE00324D55B462146179A059800F0A0
:105560004DF805441CE00498002807DBDDE9030141
:10557000884203DD0098405C179901E017993020BC
:105580005A469047049805F10105401C0490019883
:10559000401E019004D12E205A46179990476D1C49
:1055A000BAF10001AAF1010ADDDC05E017F8010BF0
:1055B0005A46179990476D1CB8F10001A8F10108EF
:1055C000F4DC5B462146179A0598ABE62D000000F7
:1055D0002B000000200000002DE9F04104460025CA
:1055E0001E461746880404D405E039462020B047FB
:1055F0006D1C641EF9D52846BDE8F0812DE9F04107
:10560000044600251E469046C80301D5302700E019
:105610002027880404D505E041463846B0476D1C74
:10562000641EF9D52846BDE8F0810A68531C0B605A
:10563000107070470000000000000000002F000004
:1056400000000700070000147F147F1400242A7F45
:105650002A120062640813230036495522500000C4
:105660000503000000001C224100000041221C0034
:105670000014083E08140008083E0808000000A0B6
:1056800060000008080808080000606000000020B2
:1056900010080402003E5149453E0000427F400090
:1056A000004261514946002141454B310018141216
:1056B0007F10002745454539003C4A4949300001E3
:1056C0007109050300364949493600064949291E32
:1056D0000000363600000000563600000008142294
:1056E0004100001414141414000041221408000294
:1056F0000151090600324959513E007C1211127CB9
:10570000007F49494936003E41414122007F4141E5
:10571000221C007F49494941007F09090901003ED7
:105720004149497A007F0808087F0000417F410015
:10573000002040413F01007F08142241007F40408B
:105740004040007F020C027F007F0408107F003E73
:105750004141413E007F09090906003E4151215E59
:10576000007F091929460046494949310001017F56
:105770000101003F4040403F001F2040201F003FEC
:105780004038403F0063140814630007087008079E
:1057900000615149454300007F41410000552A55B1
:1057A0002A55000041417F0000040201020400402C
:1057B000404040400000010204000020545454784E
:1057C000007F48444438003844444420003844446E
:1057D000487F00385454541800087E09010200180C
:1057E000A4A4A47C007F080404780000447D400049
:1057F000004080847D00007F102844000000417F2D
:105800004000007C04180478007C08040478003808
:105810004444443800FC242424180018242418FC90
:10582000007C0804040800485454542000043F44F9
:105830004020003C4040207C001C2040201C003CBC
:105840004030403C004428102844001CA0A0A07C0C
:10585000004464544C441414141414140000000044
:10586000000000000000000000000000000000F840
:1058700000000000000000333000000000100C06A3
:10588000100C0600000000000000000040C078403E
:10589000C0784000043F04043F040400007088FC0A
:1058A00008300000001820FF211E0000F008F00062
:1058B000E018000000211C031E211E0000F00888D3
:1058C000700000001E2123241927211010160E003D
:1058D000000000000000000000000000000000E0E8
:1058E00018040200000000071820400000020418FD
:1058F000E00000000040201807000000404080F059
:10590000804040000202010F01020200000000F08E
:10591000000000000101011F010101000000000062
:105920000000000080B070000000000000000000D7
:105930000000000000010101010101010000000060
:1059400000000000003030000000000000000000F7
:1059500080601804006018060100000000E01008D4
:105960000810E000000F102020100F00001010F8A9
:10597000000000000020203F2020000000700808E8
:105980000888700000302824222130000030088868
:10599000884830000018202020110E000000C02090
:1059A00010F8000000070424243F240000F80888B1
:1059B000880808000019212020110E0000E010883E
:1059C00088180000000F112020110E000038080870
:1059D000C83808000000003F000000000070880880
:1059E00008887000001C222121221C0000E0100801
:1059F0000810E0000000312222110F00000000C05A
:105A0000C0000000000000303000000000000080F6
:105A100000000000000080600000000000008040E6
:105A200020100800000102040810200040404040FF
:105A30004040400004040404040404000008102052
:105A40004080000000201008040201000070480897
:105A50000808F0000000003036010000C030C828FF
:105A6000E810E0000718272423140B000000C038BA
:105A7000E0000000203C23020227382008F8888834
:105A800088700000203F202020110E00C030080840
:105A900008083800071820202010080008F8080817
:105AA0000810E000203F202020100F0008F8888810
:105AB000E8081000203F20202320180008F88888DC
:105AC000E8081000203F200003000000C030080854
:105AD0000838000007182020221E020008F80800DD
:105AE0000008F808203F210101213F20000808F8A4
:105AF000080800000020203F2020000000000808C7
:105B0000F8080800C08080807F00000008F888C086
:105B100028180800203F20012638200008F8080037
:105B200000000000203F20202020300008F8F8006E
:105B3000F8F80800203F003F003F200008F830C080
:105B40000008F808203F200007183F00E010080870
:105B50000810E0000F10202020100F0008F808089F
:105B60000808F000203F210101010000E0100808B2
:105B70000810E0000F18242438504F0008F88888D7
:105B800088887000203F2000030C302000708808B7
:105B9000080838000038202121221C00180808F8C5
:105BA000080818000000203F2000000008F8080046
:105BB0000008F808001F202020201F000878880017
:105BC00000C83808000007380E010000F80800F887
:105BD0000008F800033C0700073C03000818688031
:105BE0008068180820302C03032C30200838C800A7
:105BF000C83808000000203F2000000010080808F6
:105C0000C83808002038262120201800000000FE97
:105C1000020202000000007F40404000000C30C043
:105C200000000000000000010638C000000202026F
:105C3000FE000000004040407F0000000000040221
:105C4000020204000000000000000000000000004C
:105C5000000000008080808080808080000202043C
:105C60000000000000000000000000000000808034
:105C7000808000000019242222223F2008F80080A2
:105C800080000000003F112020110E000000008065
:105C900080800000000E11202020110000000080F4
:105CA0008088F800000E112020103F200000808026
:105CB00080800000001F222222221300008080F03A
:105CC000888888180020203F202000000000808065
:105CD00080808000006B94949493600008F80080AA
:105CE00080800000203F210000203F200080989805
:105CF000000000000020203F202000000000008065
:105D00009898000000C08080807F000008F80000A4
:105D100080808000203F24022D302000000808F8F9
:105D2000000000000020203F2020000080808080B4
:105D300080808000203F20003F20003F8080008046
:105D400080800000203F210000203F200000808054
:105D500080800000001F202020201F008080008005
:105D60008000000080FFA12020110E0000000080B4
:105D700080808000000E112020A0FF8080808000A5
:105D80008080800020203F212000010000008080D2
:105D9000808080000033242424241900008080E0C7
:105DA000808000000000001F202000008080000094
:105DB00000808000001F202020103F208080800075
:105DC0000080808000010E30080601008080008085
:105DD000008080800F300C030C300F0000808000AA
:105DE000808080000020312E0E31200080808000D5
:105DF0000080808080818E70180601000080808085
:105E0000808080000021302C222130000000000022
:105E1000807C020200000000003F404000000000C3
:105E2000FF00000000000000FF0000000002027CF4
:105E3000800000000040403F00000000000601011B
:105E400002020404000000000000000057617465B5
:105E5000725F74656D703A25302E3166E284832C52
:105E6000207461726765743A2564E284832C207320
:105E7000657454656D703A256420E284832C207724
:105E8000617465725F6C6576656C3A25302E32669A
:105E9000636D2C2054696D6572466C61673A2564A8
:105EA000202C20486F74466C61673A25640D0A0007
:105EB000D05E0008000000208C010000D64C0008D5
:105EC000945F00088C010020BC050000684D0008AC
:105ED000071022042719172094A24A04001912015E
:105EE0000203040607080900101010FF109008882C
:105EF0008888FF888888080010130444827F018006
:105F00008040432C10284681800E1310101010D0B2
:105F100030FF30D0121C101036100804020132FF7E
:105F2000061401020408100D13FE222222FE00FEB8
:105F3000828292A29E2880601F0242827F0814FF04
:105F4000402F102C43800B1590884C57A424545498
:105F50008C8400101301018042221A0702428242FF
:105F60003E0101010E1504E4242CB4252624B42C92
:105F700024E4040C25FF02011E1212121E41827F2E
:105F80003011010203040102030406070809020498
:045F900006080000FF
:04000005080000ED02
:00000001FF
